:020000040000fa
:080000000001040000000000f3
:020000040000fa
:100200000fe8200000ff200000018800000000002f
:100210000c000700606f20000100200011000700a3
:10022000000020000000e000020032000000020098
:10023000000000000c040200000000000040da0092
:100240000000fe004440a900000020000000e00083
:100250000300320000002000a00188004440a800f4
:100260000000060091018800800078000000eb008b
:1002700015003700e280400032a0b4009101ba00be
:10028000e280400032a0b4009102ba00e280400057
:1002900032a0b4000002eb00472bde00f507b200ed
:1002a000602ce10004003a000059eb008301e900f2
:1002b000fdff3e00040037006128e100010032002c
:1002c0000082eb00040007001101ba000200e00008
:1002d000e8ff3a00000006003159ba008301e90046
:1002e0000c0032002159ba008301e90008003200f5
:1002f0000400e00003003a00e280400032a0b400b5
:10030000f5ff370011d9ba008301e900faff3a007e
:100310008100e800e180400032a0b4000000060047
:020000040000fa
:0200000401f009
:04000000e4fb00001d
:020000040000fa
:0200000401f009
:04000400ff7f00007a
:020000040000fa
:0200000401f009
:040008007fff000076
:020000040000fa
:0200000401f009
:04001400ffff0000ea
:020000040000fa
:10000800140700001407000014070000140700007c
:10001800140700001407000014070000140700006c
:10002800140700001407000014070000140700005c
:10003800140700001407000014070000140700004c
:1000480014070000540600003c06000014070000d6
:10005800140700001407000014070000140700002c
:10006800140700001407000014070000140700001c
:10007800140700001407000014070000140700000c
:10008800fc0500009c06000014070000140700008f
:1000980014070000140700001407000014070000ec
:1000a80014070000140700001407000014070000dc
:1000b80014070000140700001407000014070000cc
:1000c80014070000140700001407000014070000bc
:1000d80014070000140700001407000014070000ac
:1000e800140700001407000014070000140700009c
:0800f8001407000014070000ca
:020000040000fa
:10010800140700001407000014070000140700007b
:10011800140700001407000014070000140700006b
:10012800140700001407000014070000140700005b
:10013800140700001407000014070000140700004b
:1001480014070000540600003c06000014070000d5
:10015800140700001407000014070000140700002b
:10016800140700001407000014070000140700001b
:10017800140700001407000014070000140700000b
:10018800fc0500009c06000014070000140700008e
:1001980014070000140700001407000014070000eb
:1001a80014070000140700001407000014070000db
:1001b80014070000140700001407000014070000cb
:1001c80014070000140700001407000014070000bb
:1001d80014070000140700001407000014070000ab
:1001e800140700001407000014070000140700009b
:0801f8001407000014070000c9
:020000040000fa
:100320000600fa00100798001e009000801093004d
:100330001e00900010109300808f500003003a00c0
:100340000000eb00200798001b0037001e00900003
:1003500000109300104f78001e0090008010930052
:100360001e009000f031b000808f50000600320077
:100370001e009000001093008000e8001e00900016
:1003800001109b00030037009e0090001e009000ab
:1003900001109b001e0090005032b0001040780009
:1003a0008040e9001e0090005032b0000148780003
:1003b0001e00fb00200798002e0090000080fa002d
:1003c000000006000800fa00000f7800214798009e
:1003d0001e007800901093001e007800f031b000ed
:1003e000808f500017003a001e00780080109300a4
:1003f0001e007800808f500003003a000000eb00e0
:10040000200798002a0037001e0078001010930083
:10041000ae409000014878009e0078001e007800f1
:1004200011109b001e0078005032b0001040780080
:100430008040e8001e0078005032b000014878008b
:100440001a0037001e007800901093001e007800fc
:10045000001093000000e900808f500003003a0074
:100460000000eb0020079800110037001e00780004
:1004700010109300ae409000014878001e007800f4
:10048000101093008000e8001e00780011109b00ff
:100490001e0078005032b000104078008040e80024
:1004a0001e0078005032b00001487800020037008a
:1004b0002e009000300798003e0090000080fa0067
:1004c000000006000800fa00000f7800214798009d
:1004d0001e007800801093001e007800808f50006e
:1004e00013003a001e007800901093001e00780060
:1004f000f031b000808f500003003a000000eb00a4
:10050000200798001e0037001e007800f1312000ff
:10051000808040001e00780001109b001e007800c3
:1005200000109300ae40900001487800130037009f
:100530001e007800901093001e00780000109300b9
:100540000000e900808f500003003a000000eb003b
:10055000200798000a0037001e0078000010930062
:100560008000e9001e00780001109b001e0078004a
:1005700000109300ae409000014878000200370060
:100580002e009000300798003e0090000080fa0096
:10059000000006000400fa00000f78001e0078003a
:1005a000901093001e007800f031b000808f500052
:1005b0000b003a001e007800801093001e007800a7
:1005c000808f500003003a001000200010079800b0
:1005d0000f0037000000eb00100798000c003700f8
:1005e0001e007800901093001e0078000010930009
:1005f0000000e900808f500003003a001000200046
:1006000010079800020037000000eb001007980068
:100610001e0090000080fa00000006000a00fa00a8
:1006200020079800310798003e0090003cff07002b
:10063000204798002e009000500090000000e0003d
:1006400022003a00ae40900000c8b30080cf5000b6
:10065000080032002e009000300090008000e8007a
:100660002e009000310098000000eb004007980039
:1006700066003700ae00900000c8b30080487800e4
:10068000ae00900010002000e00098002e009000c6
:10069000500090008000e8002e009000510098006b
:1006a0002e009000500090000000e900ae00900085
:1006b0006e00400001004000ae409000014878000c
:1006c0001000200040079800500037002e009000d6
:1006d000500090008000e8002e009000510098002b
:1006e0002e009000500090000000e900ae00900045
:1006f0006e00400001004000ae40900001487800cc
:100700002e00900050009000e40f500009003c00c3
:100710002e009000904078002e40900080c0400055
:100720002e0090000148780010002000400798003b
:10073000360037002e00900050009000e50f50006a
:100740001e003a002e009000104078008080fb00d0
:1007500000102000810050002e4090000080fb001f
:10076000808f50000d003a002e0090009000900005
:100770002e00900050009000808040002e009000dd
:1007800011009800ae0090000000eb00d00098002f
:1007900021002000410798001c0037002e00900027
:1007a000400090008000e8002e009000410098007a
:1007b0000000eb0040079800140037002e00900066
:1007c00050009000000fe900090037001e0078007b
:1007d000ae0090006e004000010040001040780024
:1007e000804078003e00900036ff07001e0fe900b1
:1007f0001e00e000f5ff3c00ae0090000000eb00a2
:10080000d00098008000eb00410798004e00900057
:100810000080fa00000006000400fa000008200032
:10082000104088000000eb00204088000040eb00f2
:100830002bebb700608020003059880060802000da
:10084000405988000040eb0051eeb700c0b22000d4
:1008500060728800c0b22000707288000000eb0057
:10086000e07288000040eb0052eeb7000000eb00a1
:10087000a07288000000eb00b07288000000eb005e
:10088000c07288000000eb00d07288000000eb000e
:10089000f07288000040eb00304798000040eb0009
:1008a000204798000040eb001047980010c0b300ac
:1008b000004f780030e32f00301688000080eb00f6
:1008c000901688000080eb00f016880026010700d3
:1008d0000000eb0050168800501680000020a00099
:1008e000501688000000eb00f07388000900370004
:1008f000f0738000ee00400020e520008080400082
:100900000040eb0080487800f07380000000e800b1
:10091000f0738800f0738000e90f5000f4ff34009a
:1009200018c2bf00624060000004e0000100320015
:100930001822a900907380000000e80090738800de
:100940002e4090000040e800204798002500370026
:100950006180200020e5200030ff0700304798002c
:100960003e409000e24f50001e003a000040eb0075
:1009700065eeb7000040eb0066eeb7000000eb004c
:10098000f073880014003700f0738000ee00400020
:1009900020e5200000804000104078000080fb002f
:1009a00080108800030037002e4090000040e800cf
:1009b000204798000fc2bf00624060000004e000c2
:1009c000f9ff3a0010002000c0738800f073800027
:1009d0000000e800f0738800f0738000e60f50001c
:1009e000e9ff34003159800040598000808f500069
:1009f000d7ff3a000040eb0030479800c0738000fa
:100a00000000e00049003200030037002e40900053
:100a10000040e800204798000000eb00a073880029
:100a2000a07380000000e000f8ff3a000000eb0037
:100a3000c073880010002000d07388003b0037008e
:100a4000c0b2200036fe0700104798009e4090007c
:100a500000c8b30080cf500007003a001e04e00039
:100a600005003a0000c8b3006aeeb70010c0b3003a
:100a7000004f78002d00370010c0b3009e4f1000cb
:100a800005003a001e4090006beeb70020c0b30096
:100a9000004f78002500370020c0b3009e4f1000a3
:100aa00004003a001e4090006ceeb7001e4fe800b4
:100ab0001e00370030c0b3009e4f100004003a0003
:100ac0001e4090006deeb7001e4fe8001700370083
:100ad00040c0b3009e4f100004003a001e4090003a
:100ae0006eeeb7001e4fe8001000370050c0b30094
:100af0009e4f100004003a001e4090006feeb700b9
:100b00001e4fe8000900370060c0b3009e4f100080
:100b100006003a001e40900070eeb7001000200062
:100b2000c07388000040eb00004f780061728000c5
:100b300070728000808f5000c1ff3a000000eb000f
:100b4000d0738800c0738000e10f500025003a0088
:100b5000501680000020a200501688000000eb0014
:100b6000f073880011003700f1738000a0e62000c8
:100b700000804000104078000080fb00d01088000a
:100b8000030037002e4090000040e8002047980006
:100b900019c2bf00624060000004e000f9ff3a00a3
:100ba000f07380000000e800f0738800f0738000ac
:100bb000e60f5000ecff3400030037002e40900099
:100bc0000040e800204798000000eb00b073880068
:100bd000b07380000000e000f8ff3a000000eb0076
:100be000c07388000000eb00a07388000000eb00d9
:100bf000b07388004aff37003600f800809fbe00bf
:100c0000829fbe00849fbe00869fbe003400f80015
:100c100000002000a00188000200fa00100020005f
:100c2000000f780007003700e010800000e8b700f0
:100c3000018020009140780060802000e1fd0700e5
:100c4000000f780018c2bf00614060000004e0009f
:100c5000f5ff3a008700a9000080fa003400f9008f
:100c60004f03be004f02be004f01be004f00be004a
:100c70003600f90000400600801f78003400f800bc
:100c800000002000a00188000000fa0010002000f1
:100c9000a07388008540a9000080fa003400f900a4
:100ca0004f007800004006003600f800809fbe002c
:100cb000829fbe00849fbe00869fbe003400f80065
:100cc00000002000a00188000200fa0010002000af
:100cd000000f780051168000000820000080680096
:100ce00050168800070037009010800000e8b70019
:100cf0000180200091407800c0b22000b1fd0700c3
:100d0000000f78000ec2bf00614060000004e000e8
:100d1000f5ff3a008520a9000080fa003400f900b0
:100d20004f03be004f02be004f01be004f00be0089
:100d30003600f90000400600801f78003400f800fb
:100d400000002000a00188000000fa001000200030
:100d5000b07388008720a9000080fa003400f900f1
:100d60004f007800004006000000fa00f00020006c
:100d7000f01088008f00a8008f20a80019e2a800ba
:100d8000612120009140780090cfb30000c0600046
:100d900016e2b7001602a90018c2bf00f043b20065
:100da00018e2b70017e2a8001942a800c1202000ed
:100db0009140780090cfb30000c060000ce2b70013
:100dc0008d40a8008d20a8000fe2a800f0002000b0
:100dd000a01088000c02a8000d42a8000de2a80097
:0c0de0000f42a8000080fa00000006008e
:020000040000fa
:100dec006a0e000016000000020000000000000067
:100dfc0000000000000001000000000000000000e6
:100e0c0000000000000000000000000000080000ce
:0c0e1c006a06000000000000000000005a
:020000040000fa
:040e28000000fe00c8
:00000001FF
